:030000000219FDE5
:03000B000200A848
:03002B0002015D72
:03005B000202EEB0
:030073000202DBAB
:1000800002030406080C10182030406080040608A3
:100090000C10182030406080A0C00003070F1F051F
:1000A000050D050305030302C2AFC0D0C0E0206206
:1000B00014E5256009E473E525F4F58AD262D0E001
:1000C000D0D0D2AF3285268AC262E526F4603030C5
:1000D000682620720DD0E0D0D0C295C294C293D2CF
:1000E000AF32C295C294C293206F0D20650A740A84
:1000F000D5E0FDE57BF45290D0E0D0D0D2AF3275A0
:100100008A00C28DD26201F801B73068052065020D
:10011000D29501B7306805206502D29401B73068E6
:1001200005206502D29301B7D29230680A20650794
:100130007408D5E0FDD29501B7D29130680A2065E8
:10014000077408D5E0FDD29401B7D290D2923068FE
:100150000A2065077408D5E0FDD29301B7C2AFC28B
:10016000AD53E6EFC0D0C0E0D2D3D2AFC2CEE52AC5
:10017000600720744F152A21C47800790020742E5E
:10018000E580307E01F430E70278FF53DACF207E3D
:100190000343DA20307E0343DA10C2D8C271E5800F
:1001A000307E01F430E70279FFC3E89970CB30610B
:1001B00003752A18207403752A18885CD270E860C9
:1001C00003755F0020740DE52B6004152B21D443CB
:1001D000DA01C2D82070024147A85C206102C270D7
:1001E000207431C3E894F0400374F0F8E8C4540F6D
:1001F00028F87984B703024114C313C3138721205D
:100200000802C313200A06C3C898F8411428F850FE
:100210000374FFF8C3E895655003E565F88822E5A7
:100220002D54066022206B1FE536C333C333F8E537
:1002300064C313C313F9C3952240028922E825221F
:10024000F52250037522FF852224A824C3E52495B6
:10025000614002A8618825E5667002418BC3E8AA67
:10026000669A5003E8FAE4F9EAC333FBE568F45B05
:1002700029400D2567F8E56760021567400B418B43
:100280000AC3E5679A5002056778FF8826C26FC3E4
:10029000E52694F84002D26F20CF0AD0E0D0D043B8
:1002A000E610D2AD32C2CF053A7801E52A600530BA
:1002B0007402152AC3E55C94014005755F0041D1C5
:1002C000756000756900E55F2401F55F5003755F97
:1002D000FFD0E0D0D043E610D2AD32C2AF53E67FBC
:1002E0007592FA7593FFC260759104D2AF32C2AFB6
:1002F00053E6EFC2ADC0D0C0E0C0F0D2D3D2AFA8B9
:10030000FBA9FCC2D8307102615553DACF207E03BD
:1003100043DA10307E0343DA20D271E580307E016B
:10032000F420E702612C88278928A18253DACF20A4
:100330007E0343DA20307E0343DA10C2D8C2713024
:100340007402A16E7800E580307E01F430E702A1EE
:100350006E885CA15653DACF207E0343DA20307ECC
:100360000343DA10C271206102812E53DACF207E5E
:100370000343DA10307E0343DA20C2D8D2718857A3
:100380008958C3E89555F8E99556F97B007E087AB7
:1003900000C3E8948CE994005005755B00812088C7
:1003A0002178A2E6A8216055C3E894C8E9940050DA
:1003B00008E4D2E4FB7A0A61FBC3E89468E994019B
:1003C0005008E4D2E3FB7A0F61FBC3E894D0E994D0
:1003D000025008E4D2E2FB7A1E61FBC3E894A0E974
:1003E00094055008E4D2E1FB7A3C61FBC3E89498A1
:1003F000E994085008E4D2E0FB7A787E00C3E895DF
:1004000059FCE9955AFD30E70AECF42401FCEDF4BF
:100410003400FD755B00C3EC9AED9E5003755B01E3
:100420008859895A8557558558567802A156C3E888
:100430009527F8E99528F9307C02A13A307B02A192
:100440003A307A02A1332075028151E9FDE8FC813E
:1004500070E9C313F9E813F8307902A133E9C31343
:10046000F9E813F8307802A133E9C313FDE813FC6F
:0F04700020612CC3EC941CED940240028187EDB7
:10047F00701EC3EC94C850180529E5297002152980
:10048F00C3E529940A5002A16E755C00D270A16E6B
:10049F00E529600215297888E6F97400207F08782D
:1004AF0096B90302789EE624FAFEE43400FFC3EC0B
:1004BF009EFCED9FFD9208B90310A208500720760D
:1004CF0009D27681D9307602C276A2085016B903C6
:1004DF000DECF42401FCEDF43400FD0204F378007C
:1004EF007900A13AB90315EC33FCED33FDC3EC945D
:1004FF000AFCED9400FD50047C007D00C3EC94FFDA
:10050F00ED9400400678FF7900A13AEC8572F0A4D3
:10051F00C5F0A2F733F87900400302055678FF794A
:10052F0000020556E9C313F9E813F8307C0EE960B1
:10053F000278FFC3E81338F8E43400F9C3E894FFF6
:10054F00E99400400278FF885CD270206102A16EAE
:10055F00741FF4552F4BF52FC274EB7002D27475C4
:10056F002A18307403752A0A306102A1822074039D
:10057F0053DAFE207403752B06D0F0D0E0D0D0D222
:10058F00AD43E6103279010205B279030205B27963
:10059F000A0205B2791E0205B279640205B279C862
:1005AF000205B27817E4D5E0FDD8FAD9F6227A140D
:1005BF007B780205D97A107B8C0205D97A0D7BB432
:1005CF000205D97A0B7BC80205D9E573D5E0012264
:1005DF007902E4D291D5E0FDD294D5E0FDC294D555
:1005EF00E0FDC291D5E0FDE920E002D29530E002B6
:1005FF00D293E573D5E0FDE920E002C29530E00229
:10060F00C2937496D5E0FDD9C9EAF8D5E0FDD8FBC1
:10061F00DBB8D29122C37C007D0075F00005F0EAB3
:10062F0033FAEB33FB50F6EB13FBEA13FAC3E9FF94
:10063F00E8FEE89AF8E99BF95004EFF9EEF8B3EC0D
:10064F0033FCED33FDD5F0DFEDF9ECF822E889F05E
:10065F008A20D2D4F8A9F07B0030F70B7BFFF4246B
:10066F0001F8E9F43400F9E88520F0A4ADF0F8E9D9
:10067F008520F0A4AFF0FEED2EF974003FFA7C0454
:10068F00C3EA13FAE913F9E813F8DCF48BF030F747
:10069F000AE8F42401F8E9F43400F9E889F0C2D447
:1006AF00F8A9F02222C3E54113F9E54013F8C3E599
:1006BF004498F8E54599F9500CC3E89480E994FF04
:1006CF0040160206EBC3E8947FE99400500302063C
:1006DF00EB787F79000206EB788079FF8849894AA9
:1006EF0022E5492546F8E54A3547F9854A20E430A1
:1006FF000701F43548FA30E709C3EA94F0401502D0
:10070F000729C3EA940F500302072978FF79FF7A6C
:10071F000F020729780079007AF0C3E5249561501C
:10072F000AC374019524500B020747E54A20E70ED0
:10073F00020747E54A30E706884689478A48227804
:10074F00A5E6FAC3E54933F8E54A33F9D15CE93058
:10075F00E70BC3E89480E994FF4013E181C3E89469
:10076F007FE994005002E181787F7900E181788000
:10077F0079FFE820E715C3E52398F84009C3E8940B
:10078F000140030207A878010207A8E8F424012515
:10079F0023F840030207A878FF884B2278A6E6FAD1
:1007AF00A847A948D15CE930E70CC3E89401E99464
:1007BF00FF40160207DCC3E894FFE99400500302E0
:1007CF0007DC78FF79000207DC780179FFE920E781
:1007DF0015C3E54B98F84009C3E89401400302089C
:1007EF00037801020803E8F42401254BF8400302C3
:1007FF00080378FF88242278FF20692879A1E76011
:10080F0023E541601F74FF8541F0848539F0306A1C
:10081F000375F005A4F8C5F0600278FFC3E895648E
:10082F005002A864886322C3E5409440E5419401D7
:10083F00E5635003140147046002F5632202084F79
:10084F002275E890227883E6FF30EDF9A8BDA9BEA6
:10085F000570C3E57094084052757000E9FA79A0ED
:0F086F00E76044EA7007E571601B020888C3E880
:10087E0095716010E5715006600C140208940460C6
:10088E00F9020894E571F571C3946D401B7561C052
:10089E00C394044013756180C39404400B7561408A
:1008AE00C39404400375610075BB0622E561F460D4
:1008BE00020561E570B4070375BB1022743279A787
:1008CE0087F0A4C5F0A2F733F8C3E895614002A8FB
:1008DE0061882288248825882688642275400075C0
:1008EE0041F022C2AF75C820A8CCA9CDAA3A30CF0C
:1008FE00010A75C824D2AFAB3BAC3C883B893CC3E4
:10090E00E89BF8E99C206908F93066024102215CF7
:10091E00AD3D8A3DF9EA9DFA600678FF79FF2141E7
:10092E00AE3EAF3F8B3E8C3FA83BA93CC3E89EF842
:10093E00E99FF9C3E54113FBE54013FAE82AF540B8
:10094E00E93BF54150067540FF7541FF21A9AA40CC
:10095E00AB41AC40AD417E047F02C3EB9404400D2D
:10096E001E1FC3EB94084005206A021E1FC3ED1321
:10097E00FDEC13FCDEF7C3EA9CFAEB9DFBEF60097E
:10098E00C3E913F9E813F8DFF7EA28FAEB39FB8A23
:10099E00408B4150067BFF8B408B41C3EB94025042
:1009AE0002D2663069047F0321D47892E6FFC3E554
:1009BE0037948240110FC3E53794A040010FC3EF67
:1009CE00940640027F057E02E541C4540FF9E541CD
:1009DE00C454F0F8E540C4540F28F8C3E89EFAE971
:1009EE009400FB4009C3EA9402EB940050047A028F
:1009FE00E4FB414EAA40AB41EBC4FEEAC4540F4E99
:100A0E00FCC3EA9CFAEB9400FBC3E813C313F8EAA9
:100A1E0028FAEB3400FB8A408B41C3EB9402400270
:100A2E00C2667802EBC4FE7B00EAC4540F4EFAC3D2
:100A3E00EA98FA4005C3940250027A027892E6FFD1
:100A4E00306002414E855192855293D26043E680CA
:100A5E00C3E49AF8E49BF930660241DAE8FAE9FB5E
:100A6E00D3E913FDE813FC88518952C3EF94036058
:100A7E0038EF20E00DE82CF8E93DF9ECFAEDFB0239
:100A8E000AA3E828F8E939F9C3E82402F8E93400A2
:100A9E00F97AFE7BFFC3EF9403400E8A538B548882
:100AAE004D894E8C4F8D50610E885389548A4D8BD3
:100ABE004E8C4F8D503069127553F07554FF754F33
:100ACE00F07550FF7551F07552FF610EE8FAD3E8DC
:100ADE0013FC8851C3EF94036020EF20E007E82C4D
:100AEE00F8ECFA41FAE8282402F87AFEC3EF9403F0
:100AFE0040088A53884D8C4F610E88538A4D8C4F17
:100B0E00E568C3335002646BF56830600261187596
:100B1E003402D26043E680E52D54066034A840A925
:100B2E0041C3E913F9E813F8C3E913F9E813F830F0
:100B3E006904E92440F9C2AF53E67F759100C3E41E
:100B4E0098F594E499F595759104D26043E680D2B8
:100B5E00AF22D264754300752000306C03752040BF
:100B6E00020B7FD264754300752040306C037520F4
:100B7E000078017901206620E52D54066002C264DA
:100B8E007914E541C313700104F8C394144002783C
:100B9E0014306904781B791B206010E543600C301B
:100BAE006903D53404D26D812971200543E59B5428
:100BBE0040B52002811330690908C3E89940011835
:100BCE0061A620640A08C3E8994002617F61A6C24B
:100BDE0064C2AF53E67F759100306612759400754E
:100BEE0095F8759104D26043E680D2AF617FE541FE
:100BFE007EFFC3334005C3334001FEC3E49E7594AC
:100C0E0000F59561F0C3E53394015002617F3064C5
:100C1E0002617FD802812761A6C26DC2AF53E67F03
:100C2E00759100855394855495759104854D9285E3
:100C3E004E93D26043E680D2AFE52D540660082075
:100C4E006A020533020C65306D0D206C0A206407B4
:100C5E00158115810215392278003064027801E57C
:0F0C6E003775F007A4F9E5F028F5F0E9A2F013C7
:100C7D00A2F113A2F213F537C394785003753778A8
:100C8D00C3E53795384008D265C295C294C29330FA
:100C9D006002819C854F92855093D26043E68022FD
:100CAD00207D16C2AF754202D291C292306202D23D
:100CBD0093D2AF759F11020EA5C2AF754202D291AC
:100CCD00C290306202D295D2AF759F11020EA5303F
:100CDD007245207D22C2AF754203900139757B02AA
:100CED00C293D290D292306204D29481FCC291D23E
:100CFD00AF759F01020EA5C2AF7542039001397504
:100D0D007B02C295D292306204D294A11CC291D2C0
:100D1D00AF759F21020EA5207D17C2AF75420390BE
:100D2D000114C293306202D294D2AF759F01020EAC
:100D3D00A5C2AF754203900114C295306202D294E0
:100D4D00D2AF759F21020EA5207D16C2AF7542044C
:100D5D00D292C290306202D294D2AF759F21020E10
:100D6D00A5C2AF754204D290D292C292306202D225
:100D7D0094D2AF759F01020EA5307243207D20C223
:100D8D00AF754205900128757B04C294D2913062F3
:100D9D0004D295A1A4C292D2AF759F11020EA5C225
:100DAD00AF75420590014A757B01C294D2913062B4
:100DBD0004D293A1C4C290D2AF759F11020EA5208B
:100DCD007D17C2AF75420590010AC294306202D2FE
:100DDD0095D2AF759F11020EA5C2AF754205900158
:100DED001EC2943062EBD293D2AF759F11020EA545
:100DFD00207D18C2AF754206D290D292C291306258
:100E0D0002D295D2AF759F01020EA5C2AF754206F3
:100E1D00D292C291306202D293D2AF759F21020E4F
:100E2D00A5307246207D20C2AF75420190014A75F2
:100E3D007B01C295D292306204D293C14CC290D242
:100E4D00AF759F21020EA5C2AF75420190012875A5
:100E5D007B04C293D290D292306205D295020E6F6E
:100E6D00C292D2AF759F01020EA5207D17C2AF753C
:100E7D00420190011EC295306202D293D2AF759F8E
:100E8D0021020EA5C2AF75420190010AC2933062D4
:100E9D0002D295D2AF759F01C26522900108757B74
:100EAD0000C295C294C293D292D291D290C26222C4
:100EBD00788076FF0876FF0876FF0876FF087603C0
:100ECD0008760408760A0876030876010876017814
:100EDD008C76010876FF0876FF0876FF0876FF0806
:100EED0076FF0876030876FF0876FF0876FF08760A
:100EFD00250876D00876FA0876FA0876040876FF83
:100F0D0008760108760008767A0876FF08760108DB
:100F1D007601087600087603087600227887E6FFCA
:100F2D00C272BF0302D2727888E6C394036008C20E
:100F3D007DE630E102D27DC27E7889E630E102D2D3
:100F4D007EC3EF94026008758E01D273020F617536
:100F5D008E00C273227880E6149000809378A5F6F7
:100F6D007881E6149000809378A6F67886E6149042
:100F7D00008D9378A7F67886E6F539C39402500371
:100F8D00753902789CE67538FFB402037538A0B444
:100F9D00030375388278A3E61490009A93F566D111
:100FAD00A822227896E6FA7897E6FB7888E6B403CD
:100FBD0005C3EB940EFB307F047A007BFFC3EB9AE5
:100FCD00FCC3948250027C827572000572EC8572AE
:100FDD00F0A4C3E5F0947D40F222D27FF1B012056A
:100FED00A31205A37A007B007C10120599E55C2AFB
:100FFD00FA74003BFBDCF37C04C3EB13FBEA13FA3E
:10100D00DCF7FEC27F120FB022757C00757D00E506
:10101D00EF20E6037520000520903FFFE5201460CA
:10102D0006901DFF1460009304600375EF1653D9ED
:10103D00BF7581C043FF8012059475EF0643B2035F
:10104D00E5B3240220E70DF521E5E320E006852137
:10105D00B343E301120EA87580FF75A40075F190DE
:0F106D0075D47F75908775A5BF75F2BF75D500D7
:10107C0075A60175E241120EA8E4F8F6D8FD756864
:10108C0001120EBD12158A78988673753001C2AFA5
:10109C001205AD1205BD1205A31205C41205A3124B
:1010AC0005CB1205A31216B31205AD1205AD120530
:1010BC00A8C2AF757C00757D0078FA79FA30870785
:1010CC00D9FBD8F7021C00120F29120F62120FAFB6
:1010DC00120FB078988673120EA875881075890255
:1010EC0075C82475910475D84075A82275B8027519
:1010FC00E690759B80759D0075D10E75BC5875BBBF
:10110C000675BA1175E880120594D2AF12084C75A9
:10111C00360053DACF207E0343DA20307E0343DAE5
:10112C001043DA01C2D8C2711205ADD2617B037AC9
:10113C000CE55B70077A0CDB030210BD1205A320D3
:10114C0070030210BDC270E55CC3940240E1E52F50
:10115C00541F855E5DF55EB55DD5DAD5C26153DA97
:10116C00CF207E0343DA20307E0343DA10C2D8C28C
:10117C007178A2E67008D274E52F54E0F52FC27591
:10118C007529001205A8307409C3E529940A400298
:10119C00D27512059978023074027800C3E55C9818
:1011AC0040F0C2AF1205BD1205BD1205BDD2AF1283
:1011BC0005AD754C007888E6B4030241BD12059963
:1011CC00788CE6C3940150030212BDE530C3940140
:1011DC0050030212BD757CA5757DF1207435C3E5F5
:1011EC005C94FF50030212BDC2AF1205D2D2AF12F3
:1011FC0005A8C3E55C940150EFC2AF1205BD120502
:10120C009E1205BDD2AF1205A8C3E55C94FF40E960
:10121C000217387F05D27F120FB01205A8C2AFC2D9
:10122C007F120FB0AE5CC3E55C947FD2AF5002412D
:10123C00CD120594C2AF1205D2D2AFDFD8120FE790
:10124C00C3EE94057897F61205AD1216BB7F0AD241
:10125C007F120FB01205A8C2AFC27F120FB0AE5CE6
:10126C00C3E55C947FD2AF50E4120594C2AF120573
:10127C00BD12059E1205BDD2AFDFD4120FE7EE24CE
:10128C00037896F6F87997E7C39482400398500652
:10129C00E824827897F61205AD1215D81216EA12C8
:1012AC0005A8120FB0C3E55C94FF500221E10217B0
:1012BC0038757C00757D00C3E55C954C4003855CFE
:1012CC004C1205A878017988E7B403027805C3E5C8
:1012DC005C98400221C1C2AF1205D21205D2120590
:1012EC00D2D2AF1205AD753000E4F531F5320531CF
:1012FC00E531F4703F0532789AE67819146012786B
:10130C003214600D787D14600878FA14600375321D
:10131C0000C3E53298401D120EA8120594153275C3
:10132C00310078998673C2AF1205D2D2AF78988605
:10133C00731205A812059EE52A700530740201BDD2
:10134C0078012074027806C3E55C9840A17888E6A1
:10135C00C3940360031205A8E52A70030210BDC2F2
:10136C00AF120EA8E4F522F523F524F525F526F5A4
:10137C0067D2AF7885E6C333F565E4F544F545F5FA
:10138C0046F547F548F570F52CF52DF537757008D1
:10139C0075BB1012059412085030EDFDA8BDA9BE06
:1013AC00E97001F8887112085475700875BB101239
:1013BC000F29C2AF7561FF1208CA852261852262AE
:1013CC00852263D2AF75220175240175250175261E
:1013DC0001856069756A017888E6B40307C27D30BF
:1013EC007602D27DD268D269753300120DFD120ED1
:1013FC002E1208EA1208F11208EA1208F11208EA91
:10140C00120B711206B3120C66120CAD1208F1120B
:10141C000B60306E031206B42066031208063066A9
:10142C0003120836120C66120CDC1208F1120B7146
:10143C00306E031206F0120C66120D551208F112E2
:10144C000B60306E0312074E120C66120D861208DA
:10145C00F1120B71306E031207AB120C66120DFDFC
:0F146C001208F1120850120B60120C66120E2EAD
:10147B001208541208F130692F8564618564628506
:10148B006069756A0179187A0CC3E53399400CC20F
:10149B0069D26A8A357561FF0214B3C3E55C9401A6
:1014AB00400302140C021541306A25206C22E535ED
:1014BB00147006C26AD26B810CF535C3E55C9401DE
:1014CB00400302140C7888E6C394036003021541B1
:1014DB00753600788279A4E760027803C3E55F98DC
:1014EB005054307404E52A604D7888E6B403172015
:1014FB007D05207607A111307602A111206C07D251
:10150B006C856461814B78F0306C05856461782063
:10151B00C3E541985002810C306C1BC26CC27D300C
:10152B007602D27DD26A753512856461810C0536DF
:10153B00E55C6002A144753600C2AF120EA8788735
:10154B00E6FE7602120F297887EEF6E4F522F523F4
:10155B00F524F525F526F565752C00752D00D2AF14
:10156B001205A8120EA878A4E66006C292C291C218
:10157B0090307409C3E5369404400201BD41F590E7
:10158B001A0D782012161AE520B45A0CA312161A4B
:10159B00E520B4A5030215B8757CA5757DF1120E77
:1015AB00BD1215D8757C00757D000215D7901A03F6
:1015BB0078807B0A12161AA308DBF9901A0F788C25
:1015CB007B1912161AA308DBF9901A2822C2AF1244
:1015DB00165D12163A901A00740E12161FA3740998
:1015EB0012161FA3741512161F901A0378807B0A0C
:1015FB0012161EA308DBF9901A0F788C7B191216A2
:10160B001EA308DBF912167012164E901A2822E44C
:10161B0093F622E6438F01538FFDFFC3E583941CA2
:10162B00400122EF857CB7857DB7F0538FFE2243B7
:10163B008F02438F01857CB7857DB7901A0DF053D0
:10164B008FFC22901A0D745AD11F901A0E74A5D1CB
:10165B001F227A3079D07820901A40D11AE520F7E2
:10166B0009A3DAF7227A3079D0901A40E7D11F0913
:10167B00A3DAF922AB74A875BB01027984BB020211
:10168B007985BB03027986BB04027992BB0502798B
:10169B0087BB060279A3BB0702799CBB080279883A
:1016AB00BB09027989E8F7227C051205ADDCFB2228
:1016BB00C2AF1205BD1205C41205CB1205D212051D
:1016CB009E1205BD1205C41205CB1205D212059E42
:1016DB001205BD1205C41205CB1205D2D2AF22C220
:1016EB00AF1205D21205CB1205C41205BD12059E11
:1016FB001205D21205CB1205C41205BD12059E129E
:10170B0005D21205CB1205C41205BDD2AF22AE74A1
:10171B00AF75C2AF1205BD1205BD1205BD12059EF8
:10172B00DEF21205D212059EDFF8D2AF22D1BBD169
:10173B00B3D1B3757401757501757600F1197C051C
:10174B00AD5C1205ADC3ED955C70F5C3E55C940122
:10175B00400AC3E55C94FF4032021774D17FB1D8C5
:10176B00D1BBC2AF75EF16D1B3DCD50576C3E57629
:10177B009403500280C6D1B30575E5741490009F95
:10178B0093F808C3E57598500280AED1B3D1B30579
:10179B0074C3E574940A5002809C120EBDB1D8C27A
:0617AB00AF75EF16D1B38B
:0319FD00021016BF
:101A00000E0915FFFFFFFF03040A0301015AA50198
:101A1000FFFFFFFFFF03FFFFFF25D0FAFA04FF01DE
:091A2000007AFF0101000300FF40
:101A4000234F76736B794D52323041232020202072
:101A500023424C48454C4923463333302320202031
:101A60002020202020202020202020202020202076
:101C0000C2AFC2D353D9BF7581C043B20343FF8073
:101C1000752438752503B1DC7529A5752AF175E29F
:101C20004043F18053A47F75D4FFD2877DFA7803B7
:101C300079E67C10752200752300901DE97B0675FE
:101C400024987525013087028145208708D8FBD963
:101C5000F9DCF781B7308708D8FBD9F9DCF781B711
:101C6000B19CE493A3C39A6004DDC381B7DBDBB10D
:101C70008E6002812E7B08E493FAA3B16FDBF87AC1
:101C800030B16F752200752300B18EEAFCEBFDC305
:101C9000ED94FE400EB18E8A278B28ED30E0048A49
:101CA000828B83B18E7AC270D8C3ED94FE601950D6
:101CB000CEBD002BEC600F7520007521FF7529004B
:101CC000752A000200008100A827A9280809D80465
:101CD000D90281DCB192EA89AAF281CE0D81A3C337
:101CE000ED94035053EDA2E092007AC5C3E58294CF
:101CF00000E583941C508A200010438F02438F011B
:101D00008529B7852AB7F0300029A827A92808090E
:101D1000438F01538FFDD804D902A133C3E58394C7
:101D20001C4003A3A11689AAE28529B7852AB7F02A
:101D3000A3A116538FFC817F7AC1BD030CE493A34A
:101D4000FAB153DCF8B14B817F8181AA22AB23B178
:101D50006FEBFAEA6222752608C3E52313F523E543
:101D60002213F52250066323A0632201D526EAB18F
:101D7000DCB1DC75260AEAF4200102D287300102C8
:101D8000C287B1DCC3134002C201D526EB22B19257
:101D9000EAFB208702A192308702A197752608AE40
:101DA00024AF25C3EF13FFEE13FEB1E0B1DCC3EAAD
:101DB000133087024480FA30E703632201C3E5232E
:101DC00013F523E52213F52250066323A0632201B5
:101DD000D526D9E52265236523F52222AE24AF2539
:101DE0000E0FDEFEDFFCD20122424C48656C6934E6
:071DF000373164F3300601F6
:00000001FF
